:0200000480007A
:100000006F008004732F2034930F80006308FF0378
:10001000930F90006304FF03930FB0006300FF038E
:10002000130F000063040F0067000F00732F2034CC
:1000300063540F006F00400093E19153171F0000BD
:1000400023223FFC6FF09FFF732540F163100500F2
:10005000970200009382020173905230735000188F
:10006000970200009382020273905230B702008020
:100070009382F2FF7390023B9302F0017390023A75
:1000800097020000938282017390523073502030A7
:1000900073503030735040309301000097020000DD
:1000A000938282F673905230130510001315F501F8
:1000B000634C05000F00F00F930110009308D0056A
:1000C000130500007300000093020000638E02001D
:1000D00073905210B7B20000938292107390223046
:1000E00073232030E39A62F47350003097020000CB
:1000F0009382420173901234732540F173002030D3
:1001000097200000938000F01301A00A23902000A4
:1001100003970000930EA00A93012000631ED745A9
:1001200097200000938000EE37B1FFFF130101A07C
:100130002391200003972000B7BEFFFF938E0EA0EF
:1001400093013000631AD74397200000938080EB1F
:100150003711EFBE130101AA2392200003A740002C
:10016000B71EEFBE938E0EAA930140006316D741CF
:1001700097200000938000E937A1FFFF1301A10041
:100180002393200003976000B7AEFFFF938EAE006D
:10019000930150006312D73F97200000938060E7DF
:1001A0001301A00A239D20FE0397A0FF930EA00A2F
:1001B000930160006312D73D97200000938060E5B3
:1001C00037B1FFFF130101A0239E20FE0397C0FF5C
:1001D000B7BEFFFF938E0EA093017000631ED73948
:1001E000972000009380E0E237110000130101AA7C
:1001F000239F20FE0397E0FFB71E0000938E0EAAF8
:1002000093018000631AD73797200000938060E045
:1002100037A1FFFF1301A1002390200003970000E6
:10022000B7AEFFFF938EAE00930190006316D735F3
:1002300097200000938000DE37513412130181674C
:10024000138200FE2310220283920000B75E00009A
:10025000938E8E679301A0006390D23397200000A5
:10026000938040DB37310000130181099380B0FF98
:10027000A3932000172200001302E2D98312020088
:10028000B73E0000938E8E099301B0006396D22F83
:100290009301C00013020000B7D0FFFF9380D0CDC0
:1002A00017210000130101D62310110003170100CC
:1002B000B7DEFFFF938EDECD6310D72D1302120041
:1002C00093022000E31A52FC9301D00013020000B5
:1002D000B7C0FFFF9380D0CC17210000130181D25B
:1002E000130000002311110003172100B7CEFFFFF8
:1002F000938EDECC6312D7291302120093022000E2
:10030000E31852FC9301E00013020000B7C0FFFFA6
:100310009380C0BC172100001301C1CE1300000060
:10032000130000002312110003174100B7CEFFFF96
:10033000938ECEBC6312D7251302120093022000C5
:10034000E31652FC9301F00013020000B7B0FFFF68
:100350009380C0BB1300000017210000130181CA65
:100360002313110003176100B7BEFFFF938ECEBBAE
:100370006314D7211302120093022000E31852FCE9
:100380009301000113020000B7B0FFFF9380B0ABF0
:1003900013000000172100001301C1C61300000064
:1003A0002314110003178100B7BEFFFF938EBEAB6D
:1003B0006314D71D1302120093022000E31652FCAF
:1003C0009301100113020000B7E0FFFF9380B0AA71
:1003D000130000001300000017210000130181C268
:1003E000231511000317A100B7EEFFFF938EBEAADD
:1003F0006314D7191302120093022000E31652FC73
:10040000930120011302000017210000130181BF96
:10041000B720000093803023231011000317010040
:10042000B72E0000938E3E236318D71513021200D7
:1004300093022000E31A52FC9301300113020000E2
:1004400017210000130101BCB71000009380302277
:10045000130000002311110003172100B71E000034
:10046000938E3E22631AD7111302120093022000CA
:10047000E31852FC93014001130200001721000011
:10048000130141B8B7100000938020121300000040
:10049000130000002312110003174100B71E0000D3
:1004A000938E2E12631AD70D1302120093022000AE
:1004B000E31652FC930150011302000017210000C3
:1004C000130141B413000000930020112313110005
:1004D00003176100930E20116310D70B1302120053
:1004E00093022000E31C52FC930160011302000000
:1004F00017210000130101B1130000009300100147
:10050000130000002314110003178100930E100143
:100510006314D7071302120093022000E31A52FC5F
:10052000930170011302000017210000130181AD37
:100530001300000013000000B7300000938010008B
:10054000231511000317A100B73E0000938E1E0073
:100550006314D7031302120093022000E31652FC27
:1005600037C500001305F5EE97250000938585A992
:100570002393A500631030020F00F00F6380010089
:100580009391110093E111009308D00513850100A8
:10059000730000000F00F00F930110009308D005C6
:1005A0001305000073000000731000C0000000007D
:0C05B0000000000000000000000000003F
:1010000000000000000000000000000000000000E0
:1010100000000000000000000000000000000000D0
:1010200000000000000000000000000000000000C0
:1010300000000000000000000000000000000000B0
:081040000000000000000000A8
:10200000EFBEEFBEEFBEEFBEEFBEEFBEEFBEEFBE68
:10201000EFBEEFBE00000000000000000000000066
:040000058000000077
:00000001FF
